:020000040000FA
:1000000018F09FE518F09FE518F09FE518F09FE5C0
:1000100018F09FE50000A0E1F0FF1FE518F09FE554
:100020005800000040000000FC22000048000000D2
:100030004C000000000000005000000054000000D0
:10004000FEFFFFEAFEFFFFEAFEFFFFEAFEFFFFEA18
:10005000FEFFFFEAFEFFFFEAA0009FE50110A0E31C
:10006000001080E598009FE5AA10A0E35520A0E3CA
:100070002430A0E3043080E50130A0E3003080E5C7
:100080000C1080E50C2080E5083090E5013B13E280
:10009000FCFFFF0A0330A0E3003080E50C1080E590
:1000A0000C2080E55C009FE50410A0E3041080E5CF
:1000B0000210A0E3001080E54C009FE5DBF021E397
:1000C00000D0A0E1080040E2D7F021E300D0A0E199
:1000D000080040E2D1F021E300D0A0E1080040E2B6
:1000E000D2F021E300D0A0E1030C40E2D3F021E301
:1000F00000D0A0E1030C40E210009FE510FF2FE1CB
:1001000000C11FE080C01FE000C01FE0A03B004016
:1001100014010000000000EB2F0000EB2C008FE228
:10012000000C90E800A08AE000B08BE001704AE289
:100130000B005AE10000001A270000EB0F00BAE89C
:1001400018E04FE2010013E303F0471013FF2FE123
:100150006023000080230000102052E27800B028C5
:100160007800A128FBFFFF8A822EB0E13000B02882
:100170003000A12800409045004081451EFF2FE13E
:100180000030B0E30040B0E30050B0E30060B0E303
:10019000102052E27800A128FCFFFF8A822EB0E1F5
:1001A0003000A128003081451EFF2FE101C08FE201
:1001B0001CFF2FE11FB502F077F9059886460FBCAA
:1001C000009C02B07047000001C08FE21CFF2FE1CD
:1001D00030B47546AE4630BC70470000120800EBE4
:1001E0000210A0E1F0FFFFEB1CC09FE50FC08CE008
:1001F00001001CE30DE08F120FE0A0011CFF2FE1B6
:1002000001C08FE21CFF2FE102F040F85B03000009
:100210007847C046EBFFFFEB210800EB0C009FE5A1
:100220000C109FE504209FE508309FE51EFF2FE19D
:10023000803500408838004080350040EF49087024
:10024000C046EE49097D20221142FAD0704710B510
:1002500045E07D2212010021E94800680B0001F011
:10026000BFFC00283BD0E648006801F0C0FDE5492E
:1002700008600022D2430021E34800680B0001F02F
:10028000AFFC002818D0DF4800683030DF49087024
:100290004120FFF7D3FF2D20FFF7D0FFDB48007888
:1002A000FFF7CCFF0D20FFF7C9FF00221100D64851
:1002B0000068130001F045FB642000F0BCFC012045
:1002C0000004D3494861FF20F53000F0B4FC012060
:1002D0000004CF49C861FF20F53000F0ACFCB8E75E
:1002E00010B545E07D2212010021C54800680B00D1
:1002F00001F076FC00283BD0C148006801F077FD92
:10030000C04908600022D2430021BF4800680B00AA
:1003100001F066FC002818D0BA4800683030BB49AC
:1003200008704220FFF78AFF2D20FFF787FFB748AC
:100330000078FFF783FF0D20FFF780FF00221100F8
:10034000B1480068130001F0FCFA642000F073FC6F
:1003500001204004AE494861FF20F53000F06BFCFD
:1003600001204004AA49C861FF20F53000F063FC79
:10037000B8E710B545E07D2212010021A0480068D1
:100380000B0001F02DFC00283BD09D48006801F0D7
:100390002EFD9C4908600022D24300219A48006843
:1003A0000B0001F01DFC002818D096480068303082
:1003B000964908704320FFF741FF2D20FFF73EFFCD
:1003C00092480078FFF73AFF0D20FFF737FF002231
:1003D00011008D480068130001F0B3FA642000F0AA
:1003E0002AFC012080048A494861FF20F53000F092
:1003F00022FC012080048649C861FF20F53000F00E
:100400001AFCB8E710B545E07D22120100217C48B6
:1004100000680B0001F0E4FB00283BD0784800683E
:1004200001F0E5FC774908600022D24300217648BC
:1004300000680B0001F0D4FB002818D07148006858
:100440003030724908704420FFF7F8FE2D20FFF786
:10045000F5FE6E480078FFF7F1FE0D20FFF7EEFE87
:100460000022110068480068130001F06AFA642055
:1004700000F0E1FB0120C00465494861FF20F53030
:1004800000F0D9FB0120C0046149C861FF20F530AC
:1004900000F0D1FBB8E710B545E07D221201002144
:1004A000574800680B0001F09BFB00283BD05448E4
:1004B000006801F09CFC534908600022D2430021EF
:1004C000514800680B0001F08BFB002818D04D4804
:1004D000006830304D4908704520FFF7AFFE2D20F1
:1004E000FFF7ACFE49480078FFF7A8FE0D20FFF7A4
:1004F000A5FE0022110044480068130001F021FA13
:10050000642000F098FB0120000541494861FF206C
:10051000F53000F090FB012000053D49C861FF2047
:10052000F53000F088FBB8E710B50FE038480068F8
:1005300001218903084209D10022110030480068D6
:10054000130001F0FEF9C82000F075FBEEE71CB5C2
:100550000321080001F098FA29490860012001F000
:1005600082FA294908602B4829498861002088605F
:10057000012029490860832020490873452008701C
:1005800001200871032008730022009201925A2270
:1005900022A12548002300F03DF90022009201929B
:1005A0005A2222A12448002300F034F900220092AC
:1005B00001925A2221A12448002300F02BF90022A5
:1005C000009201925A2221A12348002300F022F92F
:1005D0000022009201925A2220A12348002300F019
:1005E00019F90022009201925A2220A122480023E8
:1005F00000F010F900F002FDC046FEE700C000E088
:1006000008000040000000400C00004004000040D2
:10061000008002E00000FFFF00C002E046756E634C
:1006200074696F6E410000004F02000046756E63F2
:1006300074696F6E42000000E102000046756E634F
:1006400074696F6E430000007303000046756E63AB
:1006500074696F6E440000000504000046756E6307
:1006600074696F6E450000009704000053656D5F6C
:1006700047697665000000002905000010B50024D8
:1006800006E014216143F94A881801F001F8641C5E
:10069000042CF6D3F548503000F0FAFFF3486430EC
:1006A00000F0F6FFF148783000F0F2FFEF488C30B0
:1006B00000F0EEFFED48A03000F0EAFFEB485030CC
:1006C000EB4908601430091D086010BC08BC1847CD
:1006D00010B5040001F029FCE5482C380068401CE6
:1006E000E3492C390860E3480068002808D1E14854
:1006F00004600800006801280FD1FFF7BFFF0CE07D
:10070000DB4820380068002807D1DA480068C06A52
:10071000E16A884201D8D7480460D548103800689B
:10072000401CD349103908601439E06A09688842CE
:1007300003D9CF492439E06A08601422E16A5143A1
:10074000CA4A8818211D00F0B3FF01F0F9FBC84820
:1007500020380068002807D0C6480068C06AE16AEF
:10076000884201D201F074FE10BC08BC1847FFB5E6
:1007700081B00C0015000A9E0C98006B691E890060
:10078000401800900098C008C0000090002708E0C2
:10079000E15D0C983430C155E05D002800D102E0E5
:1007A0007F1C082FF4D3C04600210C983430C1714F
:1007B000042E00D303260C98C6620C98C663002052
:1007C0000C9908640C98001D00F06FFF0C9818300D
:1007D00000F06BFF0C9800610420801B0C9988616D
:1007E0000C98406200200C99486400210C9840301D
:1007F0000172049A684603C801F030FB0C99086046
:100800000B98002802D00BA803C8016005B0F0BC0B
:1008100008BC1847FFB587B0040015001E00A800EB
:1008200001F0DBFB0700002F0DD04C2001F0D5FBC1
:1008300006900698002802D00698076305E0380065
:1008400001F024FC01E0002006900698002812D058
:1008500000220699119801AB07C3109A3300009249
:100860002A0020000899FFF782FF0698FFF730FF63
:100870000120059002E00020C043059005980BB0D0
:10088000F0BC08BC18477A4909680968002901D1F9
:10089000012100E00021002905D00021C943744A4C
:1008A0000C3A116007E072490968C968C868704A63
:1008B0000C3A41681160704710B50400206B01F0DC
:1008C000E5FB200001F0E2FB10BC08BC184770B546
:1008D000050001F02AFB002D02D16648006800E007
:1008E00028000400201D00F009FFA06A002803D0A2
:1008F0002000183000F002FF5D4810380068401CEE
:100900005B49103908605B48006884420CD1211DA6
:1009100056488C3000F0CCFE554830380068401CFA
:100920005349303908600BE051482C380068401EAC
:100930004F492C3908602000FFF7BEFFFFF7A3FFE7
:1009400001F0FEFA4A4820380068002805D04948DE
:100950000068844201D101F07BFD70BC08BC1847DF
:10096000F8B5002000904248001F006800286BD1B5
:100970003F4828380068461C3D4828380660002E4D
:100980000FD128300768001D006839490860081D2C
:10099000076018380068401C14390860FFF773FFBF
:1009A000C04633480C380068864241D3C0463048C0
:1009B00000680068002801D1012000E00020002824
:1009C00005D00020C0432A490C3908602FE0284890
:1009D0000068C068C4686568AE4203D224480C3819
:1009E000056024E0201D00F089FEA06A002803D0E5
:1009F0002000183000F082FE1D492439E06A0968A1
:100A0000884203D91A492439E06A08601422E16A4D
:100A10005143164A8818211D00F04AFE1549E06A24
:100A20000968C96A8842C2D301200090BFE7C04666
:100A300010480068C06A142148430C49085801282E
:100A400001D90120009006E009481C380068401CCC
:100A500007491C390860064818380068002801D08A
:100A6000012000900098F8BC08BC184768000040BE
:100A7000440000401000004070B50024002501F043
:100A800054FAFD480068401EFB49086008000068F1
:100A9000002856D1080028380068002851D026E0E8
:100AA000F648C068C4682000183000F027FE201DFA
:100AB00000F024FEF0492039E06A0968884203D931
:100AC000ED492039E06A08601422E16A5143EB4A9B
:100AD000783A8818211D00F0EBFDE949E06A0968C1
:100AE000C96A884203D30120E34914390860E34806
:100AF0000068002801D1012000E000200028CFD0AC
:100B0000002C01D0FFF7BFFEDB4818380668002E26
:100B10000FD0C046FFF724FF002803D00120D6499C
:100B200014390860761E002EF4D10020D2491839FD
:100B30000860D14814380068002802D0012501F06F
:100B400087FC01F0FDF9280070BC08BC1847F8B517
:100B500004000D00C84824380768C9480068001D13
:100B600000F0CCFD601C09D1002D07D0C4480168FD
:100B7000091DC248283000F09BFD1EE03E19C04808
:100B800000684660BE4208D2BD480168091DBA48E7
:100B90000830006800F098FD0FE0B9480168091DB1
:100BA000B548001D006800F08FFDB34808380068A4
:100BB000864202D2B04808380660F8BC08BC184724
:100BC000AD480068401CAC4908607047FEB50400A1
:100BD0000D0000200190FFF7F3FFA74824380068BC
:100BE00000902068461920680099884208D920683A
:100BF000B0420DD9009886420AD90120019007E041
:100C00002068B04202D80098864201D901200190A4
:100C100026600198002804D00099701A0021FFF77F
:100C200096FFFFF729FF0700002F01D101F010FC0C
:100C3000FEBC08BC184770B504000025002C08D085
:100C4000FFF7BEFF00212000FFF781FFFFF714FF31
:100C50000500002D01D101F0FBFB70BC08BC18475A
:100C600070B5040001F061F9002C02D184480068DD
:100C700000E020000500EE6A01F062F9300070BC6F
:100C800008BC184710B401000023002902D17C4C95
:100C9000246800E00C002200D06A10BC7047FEB54A
:100CA00004000D0000200090042D00D3032501F066
:100CB0003CF9002C02D17248006800E020000600D8
:100CC000F76BAF424CD0BD420BD96D4800688642ED
:100CD0000DD06B480068C06AA84208D80120009077
:100CE00005E067480068864201D101200090F06A63
:100CF0000190F16AF06B884200D1F562F563B0694A
:100D0000C00FC00702D10420401BB06171691422DA
:100D100001985043594A783A8018814201D1012004
:100D200000E00020002815D0301D00F0E7FC5249FB
:100D30002039F06A0968884203D94F492039F06A9E
:100D400008601422F16A51434C4A783A8818311DE0
:100D500000F0AEFC0098002801D001F079FBC046FD
:100D600001F0EEF8FEBC08BC1847434800680028B4
:100D700004D001204049143908602BE000203E498E
:100D8000143908600C39086800E0401E1421414302
:100D90003A4A783A5158002901D1012100E0002156
:100DA0000029F2D114224243344B783BD1184A68CF
:100DB00052684A600A0008324B68934202D14A687E
:100DC00052684A604A68D2682D4B1A602A49203915
:100DD0000860C046704770B5050001F0A6F8002D08
:100DE00002D12748006800E028000400201D00F020
:100DF00085FCA06A002803D02000183000F07EFC9B
:100E0000211D1E48283000F053FC01F099F81A48C3
:100E10001C380068002805D001F087F8FFF733FD83
:100E200001F08EF816480068844215D112481C382B
:100E30000068002802D001F00BFB0DE00F482830BD
:100E400000680D4928390968884203D100200C49FF
:100E5000086001E0FFF789FF70BC08BC184710B4B8
:100E6000010000200A001100044C28345369A342F9
:100E700008D1012307E0000040000040E0000040EE
:100E8000100000400023002B11D0F94C936AA342BC
:100E900001D1012300E00023002B08D1936A002B2D
:100EA00001D1012300E00023002B00D0012010BC61
:100EB000704770B505002C00002C28D0ED48006864
:100EC000844224D001F031F82000FFF7C8FF002849
:100ED0001BD0201D00F012FCE749E06A0968884237
:100EE00002D9E549E06A08601422E16A5143E04A08
:100EF000783A8818211D00F0DBFBDE49E06A0968BA
:100F0000C96A884201D301F0A3FA01F019F870BC54
:100F100008BC1847F8B5040000252600002730005B
:100F2000FFF79DFF002825D0D34820300068002817
:100F30001BD1D049F06A0968C96A884200D30125EB
:100F4000301D00F0DBFBCC49F06A0968884202D909
:100F5000C949F06A08601422F16A5143C44A783AD8
:100F60008818311D00F0A4FB04E031001831C0489E
:100F700000F09EFB2800F8BC08BC184770B529E0BB
:100F8000FFF71EFEBA4814300068002801D1012086
:100F900000E000200500FFF76FFD002D1AD100F0E2
:100FA000C4FFB3481430C068C468201D00F0A6FB1D
:100FB000B14808380068401EAF4908390860081F6A
:100FC0000068401E091F086000F0BAFF2000FFF70C
:100FD00073FCC046A8480C3800680028D0D170BC0B
:100FE00008BC184710B5C046FFF7C8FFA0487838BE
:100FF00000680128F8D901F02BFAF5E71CB59E4AE4
:101000001C320021684606C05A229CA19D4800233C
:10101000FFF700FC0400012C0DD101F01DFAA01E09
:1010200095491831086001201439086000200839FA
:10103000086000F070FF1CBC08BC184710B501F038
:101040000BFA00208C49091D086000F06DFF10BCF0
:1010500008BC184710B500F068FF8748001F0468F7
:1010600000F06EFF200010BC08BC18470021824A27
:10107000121F1068704780480838006870470200E7
:10108000002A02D17B48006800E01000010008003F
:101090003430704770B504000D007648016818318F
:1010A000200000F011FB01212800FFF750FD70BC6B
:1010B00008BC184770B504000D0016000120C007D9
:1010C00028436C49096888616A4801681831200022
:1010D00000F0EEFA01213000FFF739FD70BC08BCCA
:1010E000184770B50400E068C5682800183000F0A3
:1010F00005FB614820300068002814D1281D00F04D
:10110000FDFA5D49E86A0968884202D95A49E86AE5
:1011100008601422E96A5143554A783A8818291D13
:1011200000F0C6FA04E029001831514800F0C0FA76
:101130005049E86A0968C96A884205D90126012030
:101140004D490C31086000E00026300070BC08BC3E
:101150001847F8B504000D000120C007284320609F
:10116000E668200000F0CAFA301D00F0C7FA4249D4
:10117000F06A0968884202D93F49F06A086014227F
:10118000F16A51433A4A783A8818311D00F090FAD2
:101190003849F06A0968C96A884205D901270120DF
:1011A00035490C31086000E000273800F8BC08BC65
:1011B000184731491031096801602F49091F096832
:1011C0004160704770B504000D0000F0AEFE2A4883
:1011D000001F02682868401C01D100261AE0264939
:1011E000103120680968884204D06068904201D8B4
:1011F00001260FE06068101A2968884209D2286821
:101200006168511A401A28602000FFF7D2FF0026BB
:1012100000E0012600F094FE300070BC08BC1847C6
:10122000012015490C310860704712490868704761
:1012300070B505002C002C0045D00E49E06A096805
:10124000C96A88423FD2A069C00FC00705D10948CA
:101250000068C06A0421081AA0611422E06A5043A1
:10126000034A783A8018616981420DD101200CE06F
:10127000E0000040100000402000004049444C4580
:1012800000000000E50F00000020002817D0201DFE
:1012900000F034FAFB480068C06AE062FA49E06A8C
:1012A0000968884202D9F849E06A08601422E16AB4
:1012B0005143F64A8818211D00F0FAF903E0F1487D
:1012C0000068C06AE06270BC08BC184770B50400D2
:1012D00025000026002C23D0286C401E2864E96BD2
:1012E000E86A88421CD0286C002819D1281D00F01B
:1012F00005FAE86BE8620421E86A081AA861E24985
:10130000E86A0968884202D9DF49E86A086014225D
:10131000E96A5143DD4A8818291D00F0C9F9012600
:10132000300070BC08BC1847D64909688869D5499F
:101330000968C96A0422511AD24A12689161704739
:10134000D0480068002806D0CE490968080040301F
:10135000096C491C0160CB480068704770B50400F7
:101360000E0000F0E2FDC7480068406C00280BD179
:101370000121C448006840300172002E04D03000C2
:10138000FFF7E5FB01F064F800F0DAFD00F0CDFDB9
:10139000BC480068456C002D0AD0002C04D0002009
:1013A000B8490968486403E0681EB649096848649A
:1013B0000021B44800684030017200F0C1FD2800EF
:1013C00070BC08BC1847FFB581B004000D001600C2
:1013D00000F0ABFDAB4800684030007A022813D023
:1013E000A849096808004430496CA1430160012103
:1013F000A4480068403001720498002804D0049882
:10140000FFF7A5FB01F024F800F09AFD00F08DFD38
:10141000002E03D09B480068406C306099480068FB
:101420004030007A012801D1002707E0954909687A
:1014300008004430496CA94301600127002191480C
:1014400000684030017200F07BFD380005B0F0BC50
:1014500008BC1847FFB583B004000D001E00012032
:101460000290270000F061FD002E01D0786C306002
:101470004820C05D019002214820C155059B01F024
:1014800001F8051604080C0E1700786C28437864E0
:101490000EE0786C401C78640AE07D6408E00198F6
:1014A000022801D07D6401E00020029000E0C046E7
:1014B000C046019801281AD1381D00F01FF9724961
:1014C000F86A0968884202D96F49F86A08601422EC
:1014D000F96A51436D4A8818391D00F0E9F86949E5
:1014E000F86A0968C96A884201D900F0B1FF00F0C2
:1014F00027FD029807B0F0BC08BC1847FFB583B0C1
:1015000004000D001E000120019027000020009023
:10151000002E01D0786C30604820C05D029002211E
:101520004820C155059B00F0ADFF051604080C0EC0
:101530001700786C284378640EE0786C401C78645F
:101540000AE07D6408E00298022801D07D6401E091
:101550000020019000E0C046C046029801282FD12B
:10156000494820300068002813D1381D00F0C6F823
:101570004549F86A0968884202D94349F86A08600F
:101580001422F96A5143414A8818391D00F090F835
:1015900005E0390018313D48783000F089F83949C4
:1015A000F86A0968C96A88420AD90C98002803D0E9
:1015B00001210C98016003E0012033490C310860DF
:1015C000019807B0F0BC08BC1847F8B504000D003E
:1015D00026000020009034004820875D02218155BC
:1015E000706C401C7064012F2DD12748203000689A
:1015F000002813D1301D00F081F82349F06A0968F2
:10160000884202D92049F06A08601422F16A5143E5
:101610001E4A8818311D00F04BF805E031001831E2
:101620001A48783000F044F81649F06A0968C96A27
:10163000884208D9002D02D00120286003E0012053
:1016400011490C310860F8BC08BC184770B504009B
:10165000002C02D10B48006800E02000050000F0DB
:1016600064FC4820405D022804D1002148204155F7
:10167000012600E0002600F063FC300070BC08BCCE
:1016800018470000100000402000004068000040A3
:101690000100083141600021C94381600100083127
:1016A000C160016100210160704700210161704744
:1016B00042684A6093688B609368596091600861E2
:1016C00003685B1C0360704710B40B685C1C01D19D
:1016D000026907E00200083200E05268546824689A
:1016E0009C42FAD954684C604C68A1608A60516091
:1016F00008610468641C046010BC704701000A693A
:101700004B6888689860081D09C85860506888420E
:1017100001D188685060002008611068401E106088
:101720001068704770B504000E00250000F0FDFB46
:10173000296CE86B4843296840182C006860002039
:10174000A8632868A860E86B401E296C4843296894
:101750004018E860FF214420415545204155002EA6
:1017600010D12869002801D1012000E000200028C4
:1017700010D128001030FFF7B4FC00280AD000F088
:1017800067FE07E028001030FFF782FF28002430B2
:10179000FFF77EFF00F0D4FB012070BC08BC1847A7
:1017A000F8B504000D001600069F002D01D13F6022
:1017B00000E03E60FC633D6401213800FFF7B2FFAA
:1017C000F8BC08BC1847F7B582B0040015000398B0
:1017D000002801D1002702E0270003984743380082
:1017E000483000F0FAFB0600002E09D030004830E7
:1017F00001902B0000962000019A0399FFF7D0FF7B
:10180000300005B0F0BC08BC184770B5040000F00B
:101810008CFB4520055714E0606A002801D10120A7
:1018200000E00020002808D120002430FFF759FCF8
:10183000002803D0FFF7F4FC00E004E0681E000677
:101840000516002DE8DCC046FF214520015500F0BB
:1018500077FB00F06AFB4420055714E0206900285C
:1018600001D1012000E0002000280BD12000103021
:10187000FFF737FC002801D0FFF7D2FC681E0006F6
:10188000051600E001E0002DE8DCC046FF21442001
:10189000015500F055FB70BC08BC184770B504003A
:1018A00000F043FBA06BE16B884201D1012500E011
:1018B000002500F045FB280070BC08BC1847F8B5AF
:1018C00004000D00160000200090A76B206C00287B
:1018D00009D1206800282ED16068FFF7F7FC00903E
:1018E0000020606027E0002E0FD12900226CA06844
:1018F00000F0FAFB216CA0684018A0606168A06845
:10190000884218D32068A06015E02900226CE068A6
:1019100000F0EAFB216CE068401AE0602168E068B2
:10192000884203D2216C6068401AE060022E02D126
:10193000002F00D07F1E781CA0630098F8BC08BC64
:101940001847FFB583B004001D0000260094C04670
:1019500000F0EBFA0098806B0099C96B884201D3C4
:10196000022D22D12A0004990098FFF7A8FF070052
:101970000098406A002801D1012000E000200028E2
:1019800008D100982430FFF7ACFB002806D000F007
:101990005FFD03E0002F01D000F05AFD00F0D0FA07
:1019A000012007B0F0BC08BC18470598002803D1F7
:1019B00000F0C6FA0020F4E7002E03D101A8FFF7DB
:1019C000F8FB012600F0BCFAFFF7FAF800F0ADFAD8
:1019D000442000990856401C03D100210098403053
:1019E0000171452100984156491C02D100984030B0
:1019F000417100F0A5FA05A901A8FFF7E3FB002853
:101A000019D10098FFF74AFF00280ED00098103037
:101A10000599FFF73FFB0098FFF7F7FEFFF72CF85B
:101A2000002895D100F014FD92E70098FFF7EDFE35
:101A3000FFF722F88CE70098FFF7E7FEFFF71CF8A6
:101A40000020AEE710B50400002C09D00020606033
:101A50002060E0600022110020001300FFF771FFFA
:101A600010BC08BC1847F8B5040001260027220066
:101A700000210120FFF7A7FE05002800FFF7E2FF85
:101A80002800F8BC08BC184770B504000D000222FD
:101A900000212000FFF797FE0600002E00D0B5635E
:101AA000300070BC08BC1847FFB583B004000D00BF
:101AB0001600009400200190009CA06BE16B88420E
:101AC00002D30698022826D14521009847562900BE
:101AD000069A0098FFF7F3FE781C13D10098406A2D
:101AE000002801D1012000E00020002810D100983A
:101AF0002430FFF7F6FA00280AD0002E08D0012083
:101B0000306005E0781C01060916009840304171EC
:101B10000120029001E000200290029807B0F0BC82
:101B200008BC1847FEB504000D00270000200290F5
:101B30003C00B86B0190F86B0199884223D945208D
:101B4000C15700910198401CB8630098401C12D105
:101B5000786A002801D1012000E00020002810D17F
:101B600038002430FFF7BDFA00280AD0002D08D035
:101B70000120286005E00098401C01060916452058
:101B8000C155012600E000263000FEBC08BC184705
:101B900070B5040000F0C9F9A06B002801D101253F
:101BA00000E0002500F0CCF9280070BC08BC184704
:101BB00070B504000D00206C00280ED0216CE06888
:101BC0004018E0606168E068884201D32068E06006
:101BD0002800226CE16800F087FA70BC08BC184746
:101BE000FFB585B004001D0000260294C04600F039
:101BF0009CF90298806B0190019800283FD00298D0
:101C0000C76806990298FFF7D3FF002D1DD10198F0
:101C1000401E0299886302980068002803D1FFF7EC
:101C20008FFB0299486002980069002801D10120C9
:101C300000E0002000281BD102981030FFF751FA75
:101C4000002815D000F004FC12E00298C76002984A
:101C5000406A002801D1012000E00020002807D1BF
:101C600002982430FFF73DFA002801D000F0F0FB85
:101C700000F066F9012009B0F0BC08BC18470798CD
:101C8000002803D100F05CF90020F4E7002E03D116
:101C900003A8FFF78EFA012600F052F9FEF790FF35
:101CA00000F043F9442002990856401C03D100215A
:101CB000029840300171452102984156491C02D1D9
:101CC00002984030417100F03BF907A903A8FFF7E3
:101CD00079FA002826D10298FFF75AFF00281BD076
:101CE00002980068002807D100F01FF9029948689F
:101CF000FFF79EFA00F024F9029824300799FFF7C5
:101D0000C9F90298FFF781FDFEF7B6FE002800D062
:101D10006DE700F09DFB6AE70298FFF776FDFEF79E
:101D2000ABFE64E70298FFF770FDFEF7A5FE029890
:101D3000FFF72EFF0028EBD000209CE7F0B585B020
:101D400004000D001600029400200390029CA06B7A
:101D50000190019800282BD044210298415600910F
:101D600029000298FFF724FF0198411E0298816321
:101D70000098401C13D102980069002801D101206D
:101D800000E00020002811D102981030FFF7A9F9D7
:101D900000280BD0002E09D00120306006E000980A
:101DA000401C01060916029840300171012700E02D
:101DB0000027380005B0F0BC08BC1847FEB5040089
:101DC0000D00009400200190009CA06B002809D019
:101DD0000098C76829000098FFF7EAFE0098C760DE
:101DE000012600E000263000FEBC08BC184770B594
:101DF000040000F09AF8A56B00F0A2F8280070BC6F
:101E000008BC184770B50400250000F08EF82C00BF
:101E1000A96BE86B461A00F093F8300070BC08BC60
:101E200018470100886B704770B504002500280032
:101E300000F02CF970BC08BC184701008A6B002A1E
:101E400001D1012000E00020704701008A6BCB6BBC
:101E50009A4201D1012000E00020704730B4030015
:101E6000001F0C1D0460001F3F4C0460001F036036
:101E7000001F3E4C0460001F3D4C0460001F3D4CA1
:101E80000460001F3C4C0460001F3C4C0460001FB9
:101E90003B4C0460001F3B4C0460001F3A4C046044
:101EA000001F3A4C0460001F394C0460001F394C7D
:101EB0000460001F64100460001F0260001F1F24E4
:101EC0000460CC07E40F03D0202504682C43046091
:101ED000001F0024046030BC704700212E4AD160EE
:101EE0002E4811008861032151615114C9681022E4
:101EF00091432B4AD1601100096910221143284AED
:101F000011612849284A11602421284A11600121C1
:101F1000214A5160704710B5FFF7DFFF00F0D0F99C
:101F2000002010BC08BC1847704710B500F094FAA8
:101F30001F480068401C1E49086010BC08BC1847B8
:101F400010B51B48006800280AD019480068401ED8
:101F50001749086008000068002801D100F088FADD
:101F600010BC08BC18470000AAAAAAAA1212121292
:101F70001111111110101010090909090808080899
:101F800007070707060606060505050504040404F9
:101F90000303030302020202004000E060EA0000C3
:101FA00000F0FFFF8823000000F1FFFF00F2FFFFB9
:101FB0004C000040494AD108C900494A116000223A
:101FC000474B5A60474A08335A6000221A6008009B
:101FD000444A42601A0002607047F8B504000020CD
:101FE0000090FEF7EDFD3E48001F0068002805D177
:101FF000FFF7E0FF01203A49091F0860002C08D0D4
:1020000008346007400F04D06007400F0821081A09
:102010000419002C34D03348844231D2304E300081
:10202000056801E02E002D686868A04202D2286889
:102030000028F7D12A480830854221D0306808307E
:102040000090286830606868001B102810D92F198C
:102050006868001B78606C607968214800E000685F
:10206000026852688A42FAD302683A600760C04642
:102070001B49083968680968081A1949083908604D
:10208000FEF7FAFC0098F8BC08BC184770B50400CD
:102090002500002C19D0083D2E00FEF791FD3500DB
:1020A00071680F4800E00068026852688A42FAD3FB
:1020B0000268326006600A49083970680968401889
:1020C000074908390860FEF7D7FC70BC08BC184700
:1020D000034808380068704770470000240100403A
:1020E00058000040F83300007847C046030052E330
:1020F0002A00009A03C010E20800000A0130D1E46F
:1021000002005CE30C2082E001C0D1940130C0E405
:102110000130D13401C0C094042042E20130C03407
:10212000033011E22700000A042052E21B00003AAB
:1021300003C031E7020053E30800000A0F00008AE1
:102140002C34A0E104C0B1E5042052E20C3C83E150
:10215000043080E4F9FFFF2A011081E20F0000EA59
:102160002C38A0E104C0B1E5042052E20C3883E130
:10217000043080E4F9FFFF2A021081E2070000EA40
:102180002C3CA0E104C0B1E5042052E20C3483E110
:10219000043080E4F9FFFF2A031081E20000A0E18F
:1021A000822FB0E10130D12401C0D1240120D144DB
:1021B0000130C02401C0C0240120C0441EFF2FE113
:1021C000704770477047000010402DE9202052E210
:1021D0000500003A1850B1E8202052E21850A0E85B
:1021E0001850B1E81850A0E8F9FFFF2A02CEB0E17C
:1021F0001850B1281850A0281800B1481800A0485D
:102200001040BDE802CFB0E10430912404308024B6
:102210001EFF2F01822FB0E1B230D1200120D14426
:10222000B230C0200120C0441EFF2FE10E50A0E1BB
:10223000180000EB05E0A0E10050B0E10D10A0E1B6
:102240000A30A0E10700C0E300D0A0E160D08DE239
:1022500020402DE9F0F7FFEB2040BDE80060A0E34F
:102260000070A0E30080A0E300B0A0E30710C1E38A
:1022700005C0A0E1C009ACE8C009ACE8C009ACE801
:10228000C009ACE801D0A0E11EFF2FE10400C04668
:10229000C0462000FDF7BCFF00009FE51EFF2FE1B8
:1022A0001C3500400C109FE51800A0E3563412EFD7
:1022B0001EFF2FE108000000260002001EFF2FE194
:1022C0007847C0466C019FE5000090E500E090E58E
:1022D00064019FE50200BEE8001080E50100BEE851
:1022E00000F06FE1FF7FDEE80000A0E13CE09EE54A
:1022F00004F05EE2000000EF1EFF2FE104E08EE23A
:1023000001002DE900204DE90000A0E104D04DE2DC
:102310000100BDE8004020E900E0A0E10100BDE8C7
:10232000FF7F4EE90000A0E13CE04EE200004FE1FB
:1023300001002EE900019FE5000090E501002EE973
:10234000F0009FE5001090E500E081E5EC009FE5DE
:102350000FE0A0E110FF2FE1D8009FE5000090E51D
:1023600000E090E5D0009FE50200BEE8001080E5A7
:102370000100BEE800F06FE1FF7FDEE80000A0E1B1
:102380003CE09EE504F05EE201002DE900204DE90D
:102390000000A0E104D04DE20100BDE8004020E9CA
:1023A00000E0A0E10100BDE8FF7F4EE90000A0E1F0
:1023B0003CE04EE200004FE101002EE978009FE58D
:1023C000000090E501002EE968009FE5001090E50F
:1023D00000E081E568009FE50FE0A0E110FF2FE13C
:1023E000000050E30200000A50009FE50FE0A0E16A
:1023F00010FF2FE10100A0E348109FE5000081E5F8
:1024000044009FE5000080E528009FE5000090E57E
:1024100000E090E520009FE50200BEE8001080E5A6
:102420000100BEE800F06FE1FF7FDEE80000A0E100
:102430003CE09EE504F05EE2100000404C000040ED
:102440006B0D000061090000004000E030F0FFFF6C
:102450007847C046A6FFFFEA7847C04600000FE174
:10246000801080E301F021E1800000E21EFF2FE1F7
:102470007847C04600000FE18000C0E300F021E192
:102480001EFF2FE17847C04601C05EE50C0053E116
:102490000100002A0330DEE7000000EA0C30DEE72E
:1024A00083C08EE01CFF2FE17847C0461EFF2FE15E
:1024B000D024000000000040680000005801000027
:1024C0003825000068000040383B00008001000013
:1024D00000000000000000000000000000000000FC
:1024E00000000000000000000000000000000000EC
:1024F00000000000000000000000000000000000DC
:1025000000000000000000000000000000000000CB
:102510000000000000000000000000000F27000085
:10252000F833000000000000000000000000000080
:082530000000000000000000A3
:0400000500000114E2
:00000001FF
